:0C0000002AC058C070C0B5C1FBCFFACFB9
:10000C00A8C1F8CFF7CF95C1F5CFF4CFF3CFF2CF8E
:10001C0072C0F0CFEFCFEECFEDCFA0BB622A392C60
:10002C0024BA20283164AB7FFF64A774777064F422
:10003C0030EFFEBB6FB0A725020001000100750177
:10004C0044000100080046000000F894EE27ECBBC9
:10005C00F1E0FBBFEBBFE5BFF8E1F1BDE1BD8DE029
:10006C00A2E0BB27ED938A95E9F780E094E0A0E647
:10007C00ED930197E9F7E8E4F0E08591959100970D
:10008C0061F0A591B59105901590BF01F001059017
:10009C000D920197E1F7FB01F0CFEFE5EDBFE4E046
:1000AC00EEBFC0E6D1E065C1AA93BA93EA93FA9386
:1000BC00EFB7EA93A4E6B1E0B2D3849B04C0A0915D
:1000CC007001A13009F402C0E1E0AFD3E991EFBFB8
:1000DC00F991E991B991A9911895EA93EFB7EA933F
:1000EC008399A6D3839903C06624E1E09E2EE991FF
:1000FC00EFBFE99118950A921A926A937A938A93B0
:10010C009A93AA93BA93EA93FA93EFB7EA937FD5AB
:10011C0004B115B1F80166277727C6D4AAE9B9E965
:10012C0089E99EE3EFD4AEE6B1E085D4ED93FC9380
:10013C00A89573D5E991EFBFF991E991B991A9917E
:10014C0099918991799169911990099018955FD538
:10015C0000E010E0E19B02C0A895FCCF6DD3FFBB83
:10016C00EEBBE09AE0980DB31127A89532C0E19B45
:10017C0002C0A895FCCFE981FA81FFBBEEBBE881F8
:10018C00EDBBE29AE19A23960895E981F070FF9312
:10019C00EF9355D3DCDFAF91BF9155D329F04FD3FB
:1001AC00EB81EA93E4DFA89551D346D3EA93DFDFE2
:1001BC0012C02DD500E010E042D3C9DFFE2FE0E0E5
:1001CC00FF93EF9343D3C3DFAF91BF91EA0FFB1FB4
:1001DC008F01F8011FD524960895E0E03CD33ED35F
:1001EC0040D3A881B981A436E0E0BE0764F0E88171
:1001FC00F981E456F040E883F983E0918001EF5FE8
:10020C0030D3A895EECFE0918001E03011F4EEE010
:10021C0028D3A881B9811A975CF0E881F9813A97C3
:10022C00E883F983E0918101EF5F18D3A895F1CFB2
:10023C00A0918101A03021F4A0918001AE3009F091
:10024C0002C0EEE00BD3A881B98111975CF0E88174
:10025C00F9813197E883F983E0918201EF5FFBD25A
:10026C00A895F1CFA0918201A03041F4A091810119
:10027C00AE3021F4A0918001AE3009F002C0EEE066
:10028C00EAD2A89516C01A9310E0183070F4E981E0
:10029C00E07811F0C69A01C0C698A895C59AC59881
:1002AC00E981EE0FE9831F5FF0CFC79AC798C69814
:1002BC00188122960895E0918401EF5FE093840108
:1002CC00A0918401A33019F4E0E0E0938401A89A92
:1002DC00A99AAA9AEFEFEA93D6DF7724EEE17E167D
:1002EC0078F4C2D2E058FE4FE081E71531F4C0D269
:1002FC00EA5DFF4FE491EA93C6DFA8957394EECFC5
:10030C00B3D2309711F4A89807C0B5D211F4A998BC
:10031C0003C0B5D209F4AA98A89508951A9310E0D1
:10032C00809B11E0819B12E0879B13E0E12F1991D8
:10033C000895C09B02C0C09801C0C09AC29B02C065
:10034C00C29801C0C29AC49B02C0C49801C0C49A8E
:10035C001895EA9398D2E2BFE0E0E3BFC098C29848
:10036C00C49897D204C0EA93E1E0E0937401E99158
:10037C001895E0E0E8BBEFEFE7BBE0E0E5BBE7E0BA
:10038C00E4BBE3E8E2BBE0E0E1BBE3BFE2BF7BD26E
:10039C00E7BDE0E0E6BDE3E1EBBDE8E8EABDE0E0A7
:1003AC00E9BDE8BDE2BDEAE0E5BDE0E0E4BDEBE1BE
:1003BC00E3BDE1E9E9BFEBB7E06CEBBFE7E0E5BF1C
:1003CC00E0ECEABFE0E0EAB9E0E8E8B9E0E0E0BF81
:1003DC00E3E0E7B9EEE8E6B9E0E0EDB9E6BFF894A2
:1003EC00C498C298C0985BD25ED261D218F4E8EC83
:1003FC007E1608F002C03CD202C0EAE0F0E0E093C6
:10040C007A01F0937B014BD257D251D218F4E8EC1D
:10041C007E1608F002C02CD202C0E8ECF0E0E093AB
:10042C007601F09377013BD24BD241D218F4E8EC31
:10043C007E1608F002C01CD201C046D2E0937801AF
:10044C00F09379012CD243D2B4DE7E2E772011F4B6
:10045C00472C02C0E1E04E2EE0E1F7E23CD2E1E0B5
:10046C008E2E17D27894A8958399E2D1A0E0839927
:10047C00A1E0A03019F4E2E09E1608F002C0662458
:10048C009924A895662049F52BD231D2DCD149F0BC
:10049C0027D2E0937E01F0937F01E2E3F0E02CD2CF
:1004AC00A895A0916401B09165011B97A8F0E0E0BC
:1004BC00E0936401E09365011AD223D2EA1BFB0B93
:1004CC001BD2A0917D01AA233AF4E1E0E0937301E1
:1004DC0018D2EC59FF4F10D2A895A0917301A130FE
:1004EC0019F4E0E0E61509F011C0A0917001A130FB
:1004FC0069F4C49AC29AC09AE0E0EFBDE3E0EEBDA5
:10050C00E2E0E3BFE0E0E09373018FD1A0917401CE
:10051C00A13091F4E0E0E0937401F50131965F01B4
:10052C00F60131966F01A2E6B1E079D1A6E6B1E011
:10053C0076D1A8E6B1E073D1ECE3F0E0EC15FD0563
:10054C0018F4CC24DD24B7DEE8E5F2E0EA15FB056F
:10055C0008F0FBC0AA24BB24E1DE5E2EE0E0E5152A
:10056C0031F4E1E0E81519F4E0E0E61509F002C019
:10057C00B7D1CCD1552091F5A2E6B1E050D1A091E4
:10058C006201B0916301A134ECE9BE0730F1E1E006
:10059C008E2EBFD1E1E0E615F1F4E92DC0D13097F4
:1005AC00C9F069D131F4E0E05CD1E1E157D1E1E18E
:1005BC000FC065D131F4E3E054D1E8E04FD1E0E075
:1005CC0007C0AFD139F4E6E14CD1E9E047D1E0E125
:1005DC00E093820102C084D199D101C09AD1E3E0A9
:1005EC00E51589F5A2D1A4D1919768F1A6D1839490
:1005FC00E6E0E81510F4E1E08E2EA5D139F4E3E144
:10060C0030D1E4E12BD1E5E126D11DC038D121F464
:10061C009DD1E8E120D117C084D121F497D1E7E135
:10062C001AD111C097D139F4E3E01BD1EDE016D10A
:10063C004092820108C092D131F4E3E012D1E6E19C
:10064C000DD1EBE108D1E1E0E51509F040C06DD129
:10065C006FD11597E0F171D176D159F483D187D14F
:10066C00AE17BF071CF4AAE7B1E0D9D039D14ED1EF
:10067C002EC005D151F480D1A83CE0E0BE071CF49B
:10068C00A6E7B1E0CCD07DD122C04BD151F46AD1D8
:10069C007CD1AE17BF071CF4A8E7B1E0C0D07AD16B
:1006AC0016C058D129F4E1E04E2E409282010FC0C1
:1006BC0055D169F4F4D0F7D071D1FED077D100D1F7
:1006CC007AD17ED1ECD003D1E42D29D179D1E2E0DD
:1006DC00E515D9F52AD12CD11597B8F12ED133D1F6
:1006EC0051F469D144D1AFD01CF4AAE7B1E06BD17D
:1006FC00F7D00CD12AC0C3D049F45DD13DD1A3D0E1
:10070C001CF4A6E7B1E05FD13CD11FC00AD141F483
:10071C003CD113971CF0A8E7B1E055D13BD115C0E3
:10072C0019D121F44424409282010FC017D169F4ED
:10073C00B6D0B9D033D1C0D039D1C2D03CD140D150
:10074C00AED0C5D0E42DEBD03BD1E1E0E41541F4C3
:10075C00A0916601B0916701A935E2E0BE0708F4EB
:10076C0023C0E0E0E0936601E0936701FBD031D158
:10077C006AD010F4F7D012C01ED12BD1AE17BF0720
:10078C0010F419D10BC0E0917A01F0917B0121D1C9
:10079C005AD041F0E0916E01F0916F01E0937A0133
:1007AC00F0937B01A895369AE0916C01F0916D0164
:1007BC00A0916801B091690146D010F5E1E0E61511
:1007CC0031F4C19B02C0C19801C0C19A01C0C19A49
:1007DC00E1E0E91519F4E0E4FFE17DD0E2E0E91590
:1007EC0019F4E0E0FDE777D0E3E0E91519F4E0E374
:1007FC00F2EF71D0E0E0E0936801E0936901A89515
:10080C00A0916A01B0916B01A939EAE3BE0728F007
:10081C00E0E0E0936A01E0936B0126CEFFCFED910F
:10082C00FD913196FE93EE930895E0937001089537
:10083C00E1E06E2E9E2E0895EA81FB810895FCDF87
:10084C00FA93EA930895EA17FB070895F5DF3196BA
:10085C00FA93EA930895E09382010895E09381015D
:10086C000895E09380010895E0918401F0E00895EB
:10087C00E72DF0E00895E130A0E0FA070895E230AA
:10088C00A0E0FA070895E0E0EFBDEEBDEDBDECBDD4
:10089C000895E0E0E0937201E0937101C6CFE0911E
:1008AC007501F0E008953296FA93EA93089581DC8D
:1008BC007E2EE1E0E71508953496FA93EA930895B5
:1008CC003696FA93EA930895E2E0F0E008953896AC
:1008DC00FA93EA930895E0936C01F0936D010895F7
:1008EC00A0917A01B0917B01EFDF7ED10895A091A8
:1008FC007E01B0917F010895E0937C01F0937D011E
:10090C000895E0917C01F0917D010895FA93EA93AA
:10091C0064CCE0E0E0936201E09363010895F0E0C1
:10092C000895E330A0E0FA070895A0E6B1E077CF90
:10093C00A0916001B09161010895E0E0E093600145
:10094C00E09361010895E82DEADF95CFE5E189DFB9
:10095C00E3E184CFE430A0E0FA070895E530A0E0AD
:10096C00FA070895E0917601F09177010895A0912E
:10097C007A01B0917B010895A0917601B091770135
:10098C000895FADFA1DF30D1C1CFA0917801B091E9
:10099C0079010895FADF98DF27D1B8CFE0917A0179
:1009AC00F0917B01FA93EA93F0DB79CFDBDFFA93DA
:1009BC00EA93EBDB74CFE0917801F0917901089523
:1009CC00FA93EA93E2CBED91FD913197FE93EE937E
:1009DC000895A0916E01B0916F010895552342F4D2
:1009EC00503811F4E0FF04C03196691F791F6BF089
:1009FC0050E8572711F45F9373C05F3F31F0660FD7
:100A0C00000C57956795752F08955F9300200AF099
:100A1C0073C06CC050E8192E1522880F991F9527AA
:100A2C00550F879550E8072E0522660F771F7527FF
:100A3C00550F67950895689401C0E8945F93F2DFB1
:100A4C00703818F07F3F08F44BC056E1571BAAF4DE
:100A5C00519558300EF4593030F0EFEFFFEF6FEF47
:100A6C007FE777F91AC077275523B9F0EE0FFF1FF0
:100A7C00661F771F5A95D1F710C07727583028F08A
:100A8C00EF2FF62F672F5850F9CF552331F076956D
:100A9C006795F795E7955A95D1F700200AF484D01D
:100AAC005F910895689401C0E8943097604070405D
:100ABC00B1F0002426F0772312F4009475D0172E91
:100ACC007EE1112032F07A95EE0FFF1F661F111C8C
:100ADC00F9CFEF2FF62F612D5F938ADF5F91089589
:100AEC00EE27FF27662777275F910895EFEFFFEF3B
:100AFC006FE77FEF5F910895EFEFFFEF6FE77FE711
:100B0C005F9108955F9386DF703851F3903841F30D
:100B1C0001240894791F23F41CF300203AF3ECCF42
:100B2C000F921F932F933F934F93112722279927AF
:100B3C00689FA0018F9F302D410D591F6B9F300D69
:100B4C00411D591F8E9F27D0BF9F25D06A9F23D050
:100B5C00BE9F1DD0AF9F1BD0AE9F110D291F391FFB
:100B6C00491F591FE32FF42F652F522F4F913F919F
:100B7C002F911F910F9066232AF0550FEE1FFF1F28
:100B8C00661F02C073954BF229DF5F910895100D1B
:100B9C00211D391F02C0200D311D491F591F0895F9
:100BAC00F195E195F0400895F09560957095E1957B
:100BBC00FF4F6F4F7F4F08956F2F660F660B762F89
:100BCC0008950024112490E1AA0FBB1F001C111CD6
:100BDC000E1A1F0A18F40E0E1F1E01C0A1609A9562
:100BEC0099F7FD01D001089504D0EBDF0EF4D8DFA6
:100BFC000895E894F7FF02C0D3DF6894B7FF06C0EE
:100C0C00A095B095119600F8039400FA08951A93E4
:100C1C000A930895198108810895099119910895ED
:00000001FF
